:1000000000308A0019290000831A0A28A500030E6F
:10001000A6000F288312A500030EA600A6140A0846
:10002000AD008A018313A50E0408A7002008A800CC
:100030002108A9002208AA002308AB002408AC006C
:1000400083128C308400001C27280C183C282708B9
:1000500084002808A0002908A1002A08A2002B0873
:10006000A3002C08A4002D088A00260E830083120A
:10007000250EA61883160900F9308F00E5308E0092
:100080000130B402B408031DAD2801303302FC3E38
:1000900003186028043EB0282E08B40060282F08FA
:1000A000B4000130B2023208930060283008B40076
:1000B00060283108B4000130B2073208930060288C
:1000C0000130B502B508031DAD280130B307330870
:1000D000053C031D6D280130B30001303302FC3EA6
:1000E0000318AB28043EB8282E08B400FF30B20035
:1000F000B408031D82280130B400B500FF308F0022
:10010000E1308E00AB282F08B400B408031D8F28FF
:100110000130B400B500FF308F00E1308E00AB2815
:100120003008B400B408031D9C280130B400B500A9
:10013000FF308F00E1308E00B201AB283108B400EF
:10014000B408031DAA280130B400B500FF308F00A9
:10015000E1308E00AB28320893000C108A1127285A
:100160000A108A100A1182074C284F28562859284D
:100170000A108A100A1182077428832890289E2862
:1001800083169B019C131C141A088312B1000130C2
:1001900083169B009C131C141A088312AE000230B5
:1001A00083169B009C131C141A088312AF000330A3
:1001B00083169B009C131C141A088312B00040295C
:1001C0003630840000080319F2280230A100A00193
:1001D000A00BE828A10BE7289730A000A00BEE2881
:1001E000800BE52800343230B600E020851CFE2864
:1001F000851DFE28051EFE28851A02293230B6000C
:10020000E020F62800340430B3003108B400B50112
:10021000F9308F00E5308E00B2019301B408031D60
:1002200018290130B400B500FF308F00E1308E0096
:10023000003484011F3083051F1383161F109F1085
:100240001F119F11073083129900713083168F00A0
:100250008312B201713083168F0083121F103B305E
:100260008316850000308312A10004389200FF300D
:1002700083169200831205110C3095009301C0285B
:100280000430B3003108B400B50185309000F93076
:100290008F00E5308E00B408031D55290130B400ED
:1002A000B500FF308F00E1308E0083160C14C03093
:1002B00083128B04051C61296430B600E0205C29A0
:1002C000412A851898290B138B138B1B642931083D
:1002D000043C031C6E290130B1077D293108053C1F
:1002E000031D75290A30B1007D293108283C031D02
:1002F0007B29B1017D290A30B107F3200321831640
:100300009B018312310883169A001C1583120B0877
:10031000A0008B13831655309D00AA309D009C14BD
:100320009C1890291C11831220088B04C0308B0468
:100330008519D0290B138B138B1B9B292E08043C8A
:10034000031CA5290130AE07B4292E08053C031D66
:10035000AC290A30AE00B4292E08283C031DB2296E
:10036000AE01B4290A30AE07F32003210130831611
:100370009B0083122E0883169A001C1583120B080B
:10038000A0008B13831655309D00AA309D009C144D
:100390009C18C8291C11831220088B04C0308B04C0
:1003A000051A082A0B138B138B1BD3292F08043C27
:1003B000031CDD290130AF07EC292F08053C031D84
:1003C000E4290A30AF00EC292F08283C031DEA2954
:1003D000AF01EC290A30AF07F32003210230831666
:1003E0009B0083122F0883169A001C1583120B089A
:1003F000A0008B13831655309D00AA309D009C14DD
:100400009C18002A1C11831220088B04C0308B0416
:10041000851A402A0B138B138B1B0B2A3008043CC4
:10042000031C152A0130B007242A3008053C031D9F
:100430001C2A0A30B000242A3008283C031D222A36
:10044000B001242A0A30B007F320032103308316B9
:100450009B008312300883169A001C1583120B0828
:10046000A0008B13831655309D00AA309D009C146C
:100470009C18382A1C11831220088B04C0308B046E
:04048000612963008B
:084200000500050005000500A2
:02400E00C430BC
:00000001FF
